:10035D007B017D207F011202A4E4750F80750E25AF
:10036D00F50DF50C751040F511751210FF7E247DFD
:0C037D00F4FC1201DFE4FD7F0102041D0E
:0704660012035DD2AF80FE1E
:0300030002047D77
:01047D00324C
:03000B0002047E6E
:01047E00324B
:0300130002047F65
:01047F00324A
:03001B000204805C
:010480003249
:03002300020303D2
:10030300C0E0C0F0C083C082C0D075D000C000C0C0
:1003130001C002C003C004C005C006C0077F0212AB
:10032300046DEF60077F0212047280137F011204D1
:100333006DEF600B7F011204721203A312040BD042
:1003430007D006D005D004D003D002D001D000D00E
:0A035300D0D082D083D0F0D0E03289
:03002B000204814B
:010481003248
:0300330002048242
:010482003247
:03003B0002048339
:010483003246
:0300430002048430
:010484003245
:03004B0002048527
:010485003244
:030053000204861E
:010486003243
:10042F00538FEFE4F59853877F53A8EF53B8EF221C
:08045E00E58F54DF4FF58F22FA
:1001DF008F0B8E0A8D098C08E598542F4510451208
:1001EF00F598E5107031FFFEFDFCAB0FAA0EA90DBF
:1001FF00A80CC31201CE700453877F22E47F01FE47
:10020F00FDFCAB0FAA0EA90DA80CC31201CE600303
:10021F000202A343878022E5C854CF4511F5C8E5F4
:10022F00117036AB0FAA0EA90DA80CAF0BAE0AAD0D
:10023F0009AC0812013CE4FB7A01F9F812013C8F7A
:10024F008DAB0FAA0EA90DA80CAF0BAE0AAD09AC62
:10025F000812013C8F8BC28E22E51164307035ABD2
:10026F000FAA0EA90DA80CAF0BAE0AAD09AC081260
:10027F00013CE4FB7A01F9F812013C8FCBAB0FAADA
:10028F000EA90DA80CAF0BAE0AAD09AC0812013CBC
:05029F008FCAD2CA2243
:030477008F992238
:03047A00AF992215
:04040B00AD07AC0687
:0D040F00EC600543980880035398F78D9921
:01041C0022BD
:1003A300E598540475F040A4AD997C002DFFEC351D
:0503B300F0FE5398FB71
:0103B8002222
:10041D00EF7004C2AC8002D2ACED7003C2BC22D22C
:02042D00BC22EF
:05046D00E5985FFF228D
:05047200EFF452982296
:1003E400E4F59AF591F5A1F59BF592F5A2F5A0F542
:0403F40090F58022DE
:1002A400EF701CEB7006EDF4529A529BBB0107ED04
:1002B400F4529AED429BEB64027043ED429A22EFB2
:1002C4006401701CEB7006EDF452915292BB01076D
:1002D400EDF45291ED4292EB64027022ED429122D0
:1002E400EF64027019EB7006EDF452A152A2BB0147
:0F02F40007EDF452A1ED42A2BB0203ED42A1229D
:10043F00EF70028D80BF01028D90BF02028DA0224E
:1003F800EF7003ED4280BF0103ED4290BF0203EDB1
:0304080042A022ED
:1003B900EF7004EDF45280BF0104EDF45290BF02D6
:0603C90004EDF452A02235
:0F044F00EF7003AF8022BF0103AF9022AFA02256
:1003CF00EF7005E5805DFF22BF0105E5905DFF221F
:0503DF00E5A05DFF2216
:030000000203896F
:1003890078FFE4F6D8FD9000007F007E01E4F0A339
:0A039900DFFCDEFA75811202046633
:1001000075F008758200EF2FFFEE33FECD33CDCCB6
:1001100033CCC58233C5829BED9AEC99E582984039
:100120000CF582EE9BFEED9AFDEC99FC0FD5F0D616
:10013000E4CEFBE4CDFAE4CCF9A88222B800C1B940
:100140000059BA002DEC8BF084CFCECDFCE5F0CB7E
:10015000F97818EF2FFFEE33FEED33FDEC33FCEBB7
:1001600033FB10D703994004EB99FB0FD8E5E4F972
:10017000FA227818EF2FFFEE33FEED33FDEC33FC5F
:10018000C933C910D7059BE99A4007EC9BFCE99A53
:10019000F90FD8E0E4C9FAE4CCFB2275F010EF2F98
:1001A000FFEE33FEED33FDCC33CCC833C810D70798
:1001B0009BEC9AE899400AED9BFDEC9AFCE899F8D3
:0E01C0000FD5F0DAE4CDFBE4CCFAE4C8F92266
:1001CE00EB9FF5F0EA9E42F0E99D42F0E89C45F087
:0101DE0022FE
:00000001FF
